:020000040800F2
:1000000000060020A102000891100008111000084D
:1000100069100008111000083D100008A302000834
:10002000A3020008A3020008A3020008FD2900089B
:10003000A3020008A3020008A3020008A30200080C
:10004000A3020008A3020008A3020008A3020008FC
:10005000A3020008A3020008853E0008B13E000884
:10006000DD3E0008093F0008353F0008A3020008F4
:10007000A3020008A3020008A3020008A3020008CC
:10008000A3020008A3020008A3020008A3020008BC
:10009000A3020008A3020008A3020008613F0008B1
:1000A000A3020008A3020008A3020008A30200089C
:1000B000A3020008A3020008A3020008A30200088C
:1000C000A3020008A3020008A3020008A30200087C
:1000D000A3020008A302000839400008A302000898
:1000E000C53F0008A3020008A3020008A3020008FD
:1000F000A3020008A3020008A3020008A30200084C
:10010000A3020008A302000861400008A30200083F
:10011000A3020008A3020008A3020008A30200082B
:10012000A3020008A3020008A3020008A30200081B
:10013000A3020008A3020008A3020008A30200080B
:10014000A3020008A3020008A3020008A3020008FB
:10015000A3020008A3020008A3020008A3020008EB
:10016000A3020008A3020008A3020008A3020008DB
:10017000A302000869350008A3020008A3020008D2
:10018000A3020008A30200084D400008A3020008D3
:10019000A3020008A3020008A3020008A3020008AB
:1001A000A3020008A3020008A3020008A30200089B
:1001B000A3020008A3020008A3020008A30200088B
:1001C000A3020008A3020008A3020008A30200087B
:1001D000A302000855350008A3020008A302000886
:1001E000A3020008A3020008A3020008A30200085B
:1001F000A3020008A3020008A3020008A30200084B
:10020000A3020008A3020008A3020008A30200083A
:10021000A3020008A3020008A3020008A30200082A
:10022000A3020008A3020008A3020008A30200081A
:10023000A3020008A3020008A3020008A30200080A
:10024000A3020008A3020008A3020008A3020008FA
:10025000A3020008A3020008A3020008A3020008EA
:10026000A3020008A3020008A3020008A3020008DA
:10027000A3020008A3020008A3020008A3020008CA
:10028000A3020008A3020008A3020008A3020008BA
:10029000A3020008A3020008A3020008A3020008AA
:1002A00002E000F000F8FEE772B63A4880F30888F2
:1002B000394880F3098839484EF60851CEF20001DA
:1002C000086040F20000CCF200004EF63471CEF22D
:1002D00000010860BFF34F8FBFF36F8F40F2000043
:1002E000C0F2F0004EF68851CEF200010860BFF374
:1002F0004F8FBFF36F8F4FF00000E1EE100A4EF604
:100300003C71CEF200010860062080F31488BFF330
:100310006F8F02F031FC02F0D3FB03F06DFB4FF066
:1003200055301F491B4A91423CBF41F8040BFAE784
:100330001C49194A91423CBF41F8040BFAE71A499B
:100340001A4A1B4B9A423EBF51F8040B42F8040B69
:10035000F8E700201749184A91423CBF41F8040BC6
:10036000FAE702F0EBFB03F0CBFB144C144DAC426C
:1003700003DA54F8041B8847F9E700F041F8114C00
:10038000114DAC4203DA54F8041B8847F9E702F038
:10039000D3BB00000006002000220020000000085F
:1003A00000000020000600208844000800220020F1
:1003B0005C220020602200206C4B0020A00200087C
:1003C000A0020008A0020008A00200082DE9F04FDA
:1003D0002DED108AC1F80CD0D0F80CD0BDEC108AED
:1003E000BDE8F08F002383F311882846A047002042
:1003F00001F0E6FEFEE701F061FE00DFFEE700002F
:1004000038B502F0E3FA30B1164B00220E211A7211
:100410005A729972DA7202F0AFFA054602F0E4FA03
:100420000446D0B9104B9D4219D001339D4241F290
:10043000883512BF044600250124002002F0A6FAE8
:100440000CB100F079F800F089FD00F031FC28468D
:1004500000F020F900F070F8F9E70025EDE7054617
:10046000EBE700BF00220020010007B008B500F054
:10047000EBFBA0F120035842584108BD07B541F2FB
:100480001203022101A8ADF8043000F0FBFB03B019
:100490005DF804FB38B5202383F311881748C3683F
:1004A0000BB101F013FF0023154A4FF47A71134882
:1004B00001F0D0FE002383F31188124C236813B19E
:1004C0002368013B2360636813B16368013B636089
:1004D0000D4D2B7833B963687BB9022000F0B8FC6E
:1004E000322363602B78032B07D163682BB902207A
:1004F00000F0AEFC4FF47A73636038BD60220020D8
:10050000950400087C23002074220020084B1870FA
:1005100003280CD8DFE800F008050208022000F0EC
:100520008DBC022000F080BC024B00225A60704754
:10053000742200207C230020F8B5504B504A1C4602
:100540001968013100F0998004339342F8D1626850
:100550004C4B9A4240F291804B4B9B6803F10063F5
:1005600003F500339A4280F08880002000F0BAFB47
:100570000220FFF7CBFF454B0021D3F8E820C3F85A
:10058000E810D3F81021C3F81011D3F81021D3F8D4
:10059000EC20C3F8EC10D3F81421C3F81411D3F8ED
:1005A0001421D3F8F020C3F8F010D3F81821C3F8C1
:1005B0001811D3F81821D3F8802042F00062C3F854
:1005C0008020D3F8802022F00062C3F88020D3F886
:1005D0008020D3F8802042F00072C3F88020D3F846
:1005E000802022F00072C3F88020D3F8803072B6E9
:1005F0004FF0E023C3F8084DD4E90004BFF34F8F58
:10060000BFF36F8F224AC2F88410BFF34F8F536934
:1006100023F480335361BFF34F8FD2F8803043F619
:10062000E076C3F3C905C3F34E335B0103EA060C5E
:1006300029464CEA81770139C2F87472F9D2203B1D
:1006400013F1200FF2D1BFF34F8FBFF36F8FBFF3C2
:100650004F8FBFF36F8F536923F40033536100232F
:10066000C2F85032BFF34F8FBFF36F8F202383F355
:100670001188854680F308882047F8BD00000208ED
:1006800020000208FFFF0108002200200044025859
:1006900000ED00E02DE9F04F93B0B44B2022FF2194
:1006A00000900AA89D6800F003FCB14A1378A3B932
:1006B0000121B0481170C360202383F31188C368FF
:1006C0000BB101F003FE0023AB4A4FF47A71A94845
:1006D00001F0C0FD002383F31188009B13B1A74BE9
:1006E000009A1A60A64A1378032B03D000231370D4
:1006F000A24A53604FF0000A009CD3465646D146AA
:10070000012000F09BFB24B19C4B1B68002B00F0E8
:100710002682002000F098FA0390039B002BF2DB66
:10072000012000F081FB039B213B1F2BE8D801A295
:1007300052F823F0B5070008DD070008710800082B
:100740000107000801070008010700080309000865
:10075000D30A0008ED0900084F0A0008770A0008CC
:100760009D0A000801070008AF0A000801070008F9
:10077000210B00085508000801070008650B000858
:10078000C107000855080008010700084F0A0008C3
:100790000107000801070008010700080107000819
:1007A0000107000801070008010700080107000809
:1007B000710800080220FFF759FE002840F0F98177
:1007C000009B022105A8BAF1000F08BF1C4641F2A8
:1007D0001233ADF8143000F055FA91E74FF47A7007
:1007E00000F032FA071EEBDB0220FFF73FFE002885
:1007F000E6D0013F052F00F2DE81DFE807F0030AB3
:100800000D1013360523042105A8059300F03AFACC
:1008100017E004215548F9E704215A48F6E7042176
:100820005948F3E74FF01C08404608F1040800F06F
:100830005BFA0421059005A800F024FAB8F12C0F0A
:10084000F2D101204FF0000900FA07F747EA0B0B3D
:100850005FFA8BFB00F078FB26B10BF00B030B2B40
:1008600008BF0024FFF70AFE4AE704214748CDE706
:10087000002EA5D00BF00B030B2BA1D10220FFF70C
:10088000F5FD074600289BD00120002600F02AFA3B
:100890000220FFF73BFE5FFA86F8404600F032FA8E
:1008A0000446B0B1039940460136A1F140025142DD
:1008B000514100F037FA0028EDD1BA46044641F222
:1008C0001213022105A83E46ADF8143000F0DAF903
:1008D00016E725460120FFF719FE244B9B68AB4223
:1008E00007D9284600F000FA013040F0678104354E
:1008F000F3E70025224BBA463E461D701F4B5D6054
:10090000A8E7002E3FF45CAF0BF00B030B2B7FF43A
:1009100057AF0220FFF7FAFD322000F095F9B0F151
:100920000008FFF64DAF18F003077FF449AF0F4AF8
:1009300008EB0503926893423FF642AFB8F5807F1B
:100940003FF73EAF124BB845019323DD4FF47A7069
:1009500000F07AF90390039A002AFFF631AF039A68
:100960000137019B03F8012BEDE700BF00220020B7
:100970007823002060220020950400087C230020BA
:100980007422002004220020082200200C220020D3
:1009900078220020C820FFF769FD074600283FF4B1
:1009A0000FAF1F2D11D8C5F120020AAB25F00300AF
:1009B00084494245184428BF4246019200F052FA49
:1009C000019AFF217F4800F073FA4FEAA803C8F3A9
:1009D00087027C492846019300F072FA06460028F7
:1009E0003FF46DAF019B05EB830533E70220FFF772
:1009F0003DFD00283FF4E4AE00F0B2F900283FF4DA
:100A0000DFAE0027B846704B9B68BB4218D91F2F3A
:100A100011D80A9B01330ED027F0030312AA134406
:100A200053F8203C05934046042205A9043700F002
:100A300031FB8046E7E7384600F056F90590F2E7CB
:100A4000CDF81480042105A800F01CF902E700236A
:100A5000642104A8049300F00BF900287FF4B0AEE1
:100A60000220FFF703FD00283FF4AAAE049800F02F
:100A70006DF90590E6E70023642104A8049300F0D3
:100A8000F7F800287FF49CAE0220FFF7EFFC002867
:100A90003FF496AE049800F05BF9EAE70220FFF716
:100AA000E5FC00283FF48CAE00F06AF9E1E7022093
:100AB000FFF7DCFC00283FF483AE05A9142000F00A
:100AC00065F907460421049004A800F0DBF83946D4
:100AD000B9E7322000F0B8F8071EFFF671AEBB0789
:100AE0007FF46EAE384A07EB0903926893423FF6F3
:100AF00067AE0220FFF7BAFC00283FF461AE27F092
:100B000003074F44B9453FF4A5AE484609F104092F
:100B100000F0EAF80421059005A800F0B3F8F1E729
:100B20004FF47A70FFF7A2FC00283FF449AE00F0C2
:100B300017F9002844D00A9B01330BD008220AA9D8
:100B4000002000F0BDF900283AD02022FF210AA899
:100B500000F0AEF9FFF792FC1C4801F037FB13B030
:100B6000BDE8F08F002E3FF42BAE0BF00B030B2BE8
:100B70007FF426AE0023642105A8059300F078F8E1
:100B8000074600287FF41CAE0220FFF76FFC80466A
:100B900000283FF415AEFFF771FC41F2883001F0F8
:100BA00015FB059800F014FA46463C4600F0CCF9D7
:100BB000A6E506464EE64FF0000901E6BA467EE697
:100BC00037467CE67822002000220020A086010023
:100BD000F7B50C46184E4FF47A71054602FB01F347
:100BE00096F90020501C0BD1144829460193026845
:100BF000176A2246B8478442019B03D1002310E0C4
:100C0000002AF1D096F90020511C01D0012A0DD103
:100C10000B4829460268166A2246B047844205D12D
:100C20000123084A0120137003B0F0BD4FF4FA709D
:100C300001F0CCFA0020F7E710220020CC2300209E
:100C4000602E0020C8230020002307B502460121A2
:100C50000DF107008DF80730FFF7BAFF20B19DF8BE
:100C6000070003B05DF804FB4FF0FF30F9E7000028
:100C70000A46042108B5FFF7ABFF80F00100C0B2BF
:100C8000404208BD074B0A4630B41978064B53F86A
:100C90002140014623682046DD69044BAC4630BC48
:100CA000604700BFC82300205C410008A086010007
:100CB00070B50A4E00240A4D01F036FD30802868D8
:100CC0003388834208D901F02BFD2B68044401339B
:100CD000B4F5003F2B60F2D370BD00BFCA230020E3
:100CE0008423002001F0FEBD00F1006000F500301B
:100CF0000068704700F10060920000F5003001F0DC
:100D000075BD0000054B1A68054B1B889B1A834272
:100D100002D9104401F004BD002070478423002054
:100D2000CA23002038B50446074D29B1286820445D
:100D3000BDE8384001F00CBD2868204401F0F6FC05
:100D40000028F3D038BD00BF842300200020704766
:100D500000F1FF5000F58F10D0F800087047000038
:100D6000064991F8243033B100230822086A81F83B
:100D70002430FFF7BFBF0120704700BF8823002049
:100D8000014B1868704700BF0010005C244BF0B5A1
:100D90001A680446234BC2F30B06120C1F885868CE
:100DA000BE4293F9085028D09F89BE4206D1012047
:100DB0000C2505FB0033586893F9085041F20103F4
:100DC0009A421CD041F203039A421AD042F2010324
:100DD0009A4218D042F203039A4208BF5625621E77
:100DE0000B46441E0A4493420FD214F9016F581C5B
:100DF0006EB1034600F8016CF5E70020D8E75A25EC
:100E0000EDE75925EBE75825E9E7184605E02C24DE
:100E100082421C7001D9981C5D70401AF0BD00BF61
:100E20000010005C14220020022803D1024B4FF076
:100E300000629A61704700BF00040258022803D183
:100E4000024B4FF400629A61704700BF00040258E1
:100E5000022804D1024A536983F400635361704746
:100E600000040258002310B5934203D0CC5CC45454
:100E70000133F9E710BD0000013810B510F9013F4A
:100E80003BB191F900409C4203D11AB10131013AC2
:100E9000F4E71AB191F90020981A10BD1046FCE74A
:100EA00003460246D01A12F9011B0029FAD17047F5
:100EB00002440346934202D003F8011BFAE770474D
:100EC0002DE9F8431F4D14460746884695F824201F
:100ED00052BBDFF870909CB395F824302BB92022D8
:100EE000FF2148462F62FFF7E3FF95F824004146B3
:100EF000C0F1080205EB8000A24228BF2246D6B20C
:100F00009200FFF7AFFF95F82430A41B17441E444E
:100F10009044E4B2F6B2082E85F82460DBD1FFF7E6
:100F20001FFF0028D7D108E02B6A03EB820383421E
:100F3000CFD0FFF715FF0028CBD10020BDE8F88304
:100F40000120FBE788230020024B1A78024B1A701D
:100F5000704700BFC82300201022002038B5164C6F
:100F6000164D204600F034FC2946204600F05CFC7B
:100F70002D681348D5F89020D2F8043843F00203C6
:100F8000C2F8043801F022F90E49284600F05AFD53
:100F9000D5F890200C48D2F804380C49A04223F030
:100FA0000203C2F804384FF461230B6003D0BDE89C
:100FB000384000F06BBB38BD602E0020684200084E
:100FC00040420F0070420008CC230020B0230020D4
:100FD00038B50B4B04461A780A4B53F822500A4B8B
:100FE0009D420CD0094B002118221846FFF760FFE4
:100FF000046001462846BDE8384000F047BB38BDD4
:10100000C82300205C410008602E0020B02300208F
:1010100000B59BB0EFF3098168226846FFF722FF15
:10102000EFF30583044B9A6BDA6A9A6A9A6A9A6AB2
:101030009A6A9A6A9B6AFEE700ED00E000B59BB0F1
:10104000EFF3098168226846FFF70CFFEFF3058391
:10105000044B9A6B9A6A9A6A9A6A9A6A9A6A9B6A23
:10106000FEE700BF00ED00E000B59BB0EFF30981A3
:1010700068226846FFF7F6FEEFF30583034B5A6BD1
:101080009A6A9A6A9A6A9A6A9B6AFEE700ED00E099
:10109000FEE7000030B50A44084D91420DD011F82A
:1010A000013B5840082340F30004013B2C4013F05F
:1010B000FF0384EA5000F6D1EFE730BD2083B8ED9E
:1010C000026843681143016003B11847704700008C
:1010D000024A136843F0C0031360704700440040A5
:1010E000024A136843F0C003136070470078004061
:1010F00037B51A4C1A4D204600F0BCFA04F1140022
:10110000009400234FF40072164900F07DF94FF46B
:101110000072154904F138000094144B00F0F6F900
:10112000134BC4E91735134C204600F0A3FA04F121
:10113000140000234FF400720F49009400F064F98A
:101140000E4B4FF400720E4904F13800009400F089
:10115000DDF90C4BC4E9173503B030BDCC230020BA
:1011600000E1F505A4240020A4280020D1100008E7
:101170000044004038240020A4260020E11000088C
:10118000A42A002000780040037C30B52B4C0029B5
:1011900018BF0C46012B11D1294B98423BD1294B4A
:1011A000D3F8E82042F40032C3F8E820D3F8102145
:1011B00042F40032C3F81021D3F810312268036ED4
:1011C000C16D03EB52038466B3FBF2F3626815044E
:1011D00042BF23F0070503F0070343EA4503CB6052
:1011E000A36843F040034B60E36843F001038B6066
:1011F00042F4967343F001030B604FF0FF330B6230
:10120000510505D512F0102214D0B2F1805F13D031
:1012100080F8643030BD0C4B9842CFD1094BD3F8E5
:10122000E82042F08042C3F8E820D3F8102142F0D1
:101230008042BFE77F23EBE73F23E9E764410008F3
:10124000CC23002000440258382400202DE9F04728
:10125000C66D05463768F4692107346219D014F069
:10126000080118BF8021E20748BF41F02001A30711
:101270004FF0200348BF41F04001600748BF41F4F0
:10128000807183F31188281DFFF71AFF002383F371
:101290001188E2050AD5202383F311884FF40071E9
:1012A000281DFFF70DFF002383F311884FF020095D
:1012B0004FF0000A14F0200838D13B0616D54FF045
:1012C000200905F1380A200610D589F31188504607
:1012D00000F050F9002836DA0821281DFFF7F0FE4B
:1012E00027F080033360002383F31188790614D537
:1012F000620612D5202383F31188D5E913239A427D
:1013000008D12B6C33B127F040071021281DFFF7BF
:10131000D7FE3760002383F31188E30618D5AA6E41
:101320001369ABB15069BDE8F047184789F31188DC
:10133000736A284695F86410194000F0B5F98AF3ED
:101340001188F469B6E7B06288F31188F469BAE7E6
:10135000BDE8F087F8B51546826804460B46AA42F8
:1013600000D28568A1692669761AB5420BD2184663
:101370002A46FFF777FDA3692B44A3612846A3689B
:101380005B1BA360F8BD0CD9AF1B18463246FFF7B4
:1013900069FD3A46E1683044FFF764FDE3683B4489
:1013A000EBE718462A46FFF75DFDE368E5E7000036
:1013B00083689342F7B50446154600D28568D4E9A0
:1013C0000460361AB5420BD22A46FFF74BFD63691B
:1013D0002B4463612846A3685B1BA36003B0F0BD88
:1013E0000DD93246AF1B0191FFF73CFD01993A46FA
:1013F000E0683144FFF736FDE3683B44E9E72A46FD
:10140000FFF730FDE368E4E710B50A440024C36148
:10141000029B8460C16002610362C0E90000C0E910
:10142000051110BD08B5D0E90532934201D182689B
:1014300082B98268013282605A1C426119700021AF
:10144000D0E904329A4224BFC368436100F0DAFE57
:10145000002008BD4FF0FF30FBE7000070B52023EF
:1014600004460E4683F31188A568A5B1A368A26956
:10147000013BA360531CA36115782269934224BFEA
:10148000E368A361E3690BB120469847002383F327
:101490001188284607E03146204600F0A3FE0028C8
:1014A000E2DA85F3118870BD2DE9F74F04460E4648
:1014B00017469846D0F81C904FF0200A8AF31188FE
:1014C0004FF0000B154665B12A4631462046FFF71E
:1014D00041FF034660B94146204600F083FE0028E4
:1014E000F1D0002383F31188781B03B0BDE8F08F9F
:1014F000B9F1000F03D001902046C847019B8BF340
:101500001188ED1A1E448AF31188DCE7C160C361BB
:10151000009B82600362C0E905111144C0E900002C
:1015200001617047F8B504460D461646202383F343
:101530001188A768A7B1A368013BA36063695A1C1F
:1015400062611D70D4E904329A4224BFE36863618A
:10155000E3690BB120469847002080F3118807E02B
:101560003146204600F03EFE0028E2DA87F311887B
:10157000F8BD0000D0E9052310B59A4201D1826878
:101580007AB982680021013282605A1C82611C781B
:1015900003699A4224BFC368836100F033FE20468A
:1015A00010BD4FF0FF30FBE72DE9F74F04460E4624
:1015B00017469846D0F81C904FF0200A8AF31188FD
:1015C0004FF0000B154665B12A4631462046FFF71D
:1015D000EFFE034660B94146204600F003FE0028B6
:1015E000F1D0002383F31188781B03B0BDE8F08F9E
:1015F000B9F1000F03D001902046C847019B8BF33F
:101600001188ED1A1E448AF31188DCE702684368EA
:101610001143016003B11847704700001430FFF711
:1016200043BF00004FF0FF331430FFF73DBF000011
:101630003830FFF7B9BF00004FF0FF333830FFF705
:10164000B3BF00001430FFF709BF00004FF0FF31B7
:101650001430FFF703BF00003830FFF763BF00000E
:101660004FF0FF323830FFF75DBF000000207047B9
:10167000FFF73EBD044B036000234360C0E9023323
:1016800001230374704700BF7C41000810B520237C
:10169000044683F31188FFF777FD022323740023A8
:1016A00083F3118810BD000038B5C36904460D46A8
:1016B0001BB904210844FFF7A9FF294604F11400CF
:1016C000FFF7B0FE002806DA201D4FF48061BDE868
:1016D0003840FFF79BBF38BD026843681143016083
:1016E00003B118477047000013B5406B00F58054F4
:1016F000D4F8A4381A681178042914D1017C02297D
:1017000011D11979012312898B4013420BD101A900
:101710004C3002F071F8D4F8A4480246019B2179BC
:10172000206800F0DFF902B010BD0000143001F0B5
:10173000F3BF00004FF0FF33143001F0EDBF0000A5
:101740004C3002F0C5B800004FF0FF334C3002F0CF
:10175000BFB80000143001F0C1BF00004FF0FF31EE
:10176000143001F0BBBF00004C3002F091B8000013
:101770004FF0FF324C3002F08BB800000020704771
:1017800010B500F58054D4F8A4381A6811780429EB
:1017900017D1017C022914D15979012352898B4038
:1017A00013420ED1143001F053FF024648B1D4F871
:1017B000A4484FF4407361792068BDE8104000F000
:1017C0007FB910BD406BFFF7DBBF00007047000022
:1017D0007FB5124B012504260446036000230574DF
:1017E00000F1840243602946C0E902330C4B0290A9
:1017F000143001934FF44073009601F005FF094B3C
:1018000004F69442294604F14C000294CDE90063A9
:101810004FF4407301F0CCFF04B070BDA441000848
:10182000C5170008E91600080A68202383F3118809
:101830000B790B3342F823004B79133342F8230022
:101840008B7913B10B3342F8230000F58053C3F8B2
:10185000A41802230374002383F311887047000047
:1018600038B5037F044613B190F85430ABB9012565
:10187000201D0221FFF730FF04F114006FF0010179
:10188000257700F0CBFC04F14C0084F854506FF045
:101890000101BDE8384000F0C1BC38BD10B50121E0
:1018A00004460430FFF718FF0023237784F85430F0
:1018B00010BD000038B504460025143001F0BCFE10
:1018C00004F14C00257701F08BFF201D84F8545063
:1018D0000121FFF701FF2046BDE83840FFF750BF68
:1018E00090F8803003F06003202B06D190F881201F
:1018F0000023212A03D81F2A06D800207047222A55
:10190000FBD1C0E91D3303E0034A42670722826727
:10191000C3670120704700BF2C22002037B500F5B7
:101920008055D5F8A4381A68117804291AD1017C99
:10193000022917D11979012312898B40134211D141
:1019400000F14C04204602F00BF858B101A92046E2
:1019500001F052FFD5F8A4480246019B2179206886
:1019600000F0C0F803B030BD01F10B03F0B550F842
:10197000236085B004460D46FEB1202383F3118811
:1019800004EB8507301D0821FFF7A6FEFB6806F172
:101990004C005B691B681BB1019001F03BFF019893
:1019A00003A901F029FF024648B1039B29462046BE
:1019B00000F098F8002383F3118805B0F0BDFB68B0
:1019C0005A691268002AF5D01B8A013B1340F1D1F5
:1019D00004F18002EAE70000133138B550F82140E5
:1019E000ECB1202383F3118804F58053D3F8A428A5
:1019F0001368527903EB8203DB689B695D6845B12C
:101A000004216018FFF768FE294604F1140001F074
:101A100029FE2046FFF7B4FE002383F3118838BD6A
:101A20007047000001F01CB901234022002110B5CD
:101A3000044600F8303BFFF73BFA0023C4E90133CA
:101A400010BD000010B52023044683F31188242222
:101A5000416000210C30FFF72BFA204601F022F9FB
:101A600002232370002383F3118810BD70B500EBAF
:101A70008103054650690E461446DA6018B11022FB
:101A80000021FFF715FAA06918B110220021FFF715
:101A90000FFA31462846BDE8704001F015BA000043
:101AA00083682022002103F0011310B504468360EF
:101AB0001030FFF7FDF92046BDE8104001F090BA64
:101AC000F0B4012500EB810447898D40E4683D4373
:101AD000A469458123600023A2606360F0BC01F02B
:101AE000ADBA0000F0B4012500EB810407898D40F8
:101AF000E4683D436469058123600023A26063605C
:101B0000F0BC01F023BB000070B5022300250446A1
:101B1000242203702946C0F888500C3040F8045C39
:101B2000FFF7C6F9204684F8705001F061F9636848
:101B30001B6823B129462046BDE87040184770BD98
:101B4000037880F88C300523037043681B6810B558
:101B500004460BB1042198470023A36010BD000088
:101B600090F88C20436802701B680BB10521184760
:101B70007047000070B590F87030044613B1002330
:101B800080F8703004F18002204601F04DFA63685D
:101B90009B68B3B994F8803013F0600535D000210C
:101BA000204601F0F7FC0021204601F0E7FC6368C5
:101BB0001B6813B1062120469847062384F870302D
:101BC00070BD204698470028E4D0B4F88630A26F54
:101BD0009A4288BFA36794F98030A56F002B4FF01D
:101BE000200380F20381002D00F0F280092284F8A6
:101BF000702083F3118800212046D4E91D23FFF7CC
:101C000071FF002383F31188DAE794F8812003F051
:101C10007F0343EA022340F20232934200F0C58080
:101C200021D8B3F5807F48D00DD8012B3FD0022BAF
:101C300000F09380002BB2D104F188026267022287
:101C4000A267E367C1E7B3F5817F00F09B80B3F53E
:101C5000407FA4D194F88230012BA0D1B4F8883011
:101C600043F0020332E0B3F5006F4DD017D8B3F55F
:101C7000A06F31D0A3F5C063012B90D863682046D4
:101C800094F882205E6894F88310B4F88430B047EA
:101C9000002884D0436863670368A3671AE0B3F53C
:101CA000106F36D040F6024293427FF478AF5C4B1F
:101CB00063670223A3670023C3E794F88230012BF4
:101CC0007FF46DAFB4F8883023F00203A4F88830B5
:101CD000C4E91D55E56778E7B4F88030B3F5A06F27
:101CE0000ED194F88230204684F88A3001F0DEF874
:101CF00063681B6813B101212046984703232370B2
:101D00000023C4E91D339CE704F18B0363670123BF
:101D1000C3E72378042B10D1202383F311882046B6
:101D2000FFF7BEFE85F311880321636884F88B50AA
:101D300021701B680BB12046984794F88230002B25
:101D4000DED084F88B300423237063681B68002B7B
:101D5000D6D0022120469847D2E794F88430204616
:101D60001D0603F00F010AD501F050F9012804D037
:101D700002287FF414AF2B4B9AE72B4B98E701F026
:101D800037F9F3E794F88230002B7FF408AF94F82A
:101D9000843013F00F01B3D01A06204602D501F0AB
:101DA00011FCADE701F002FCAAE794F88230002BA9
:101DB0007FF4F5AE94F8843013F00F01A0D01B0629
:101DC000204602D501F0E6FB9AE701F0D7FB97E742
:101DD000142284F8702083F311882B462A46294662
:101DE0002046FFF76DFE85F31188E9E65DB1152207
:101DF00084F8702083F3118800212046D4E91D2344
:101E0000FFF75EFEFDE60B2284F8702083F3118855
:101E10002B462A4629462046FFF764FEE3E700BF2B
:101E2000D4410008CC410008D041000838B590F8F2
:101E300070300446002B3ED0063BDAB20F2A34D86D
:101E40000F2B32D8DFE803F037313108223231313D
:101E50003131313131313737856FB0F886309D42BD
:101E600014D2C3681B8AB5FBF3F203FB12556DB99C
:101E7000202383F311882B462A462946FFF732FE9A
:101E800085F311880A2384F870300EE0142384F857
:101E90007030202383F31188002320461A46194608
:101EA000FFF70EFE002383F3118838BDC36F03B123
:101EB00098470023E7E70021204601F06BFB002153
:101EC000204601F05BFB63681B6813B106212046C6
:101ED00098470623D7E7000010B590F87030044605
:101EE000142B29D017D8062B05D001D81BB110BD53
:101EF000093B022BFBD80021204601F04BFB0021BF
:101F0000204601F03BFB63681B6813B106212046A5
:101F10009847062319E0152BE9D10B2380F8703080
:101F2000202383F3118800231A461946FFF7DAFDB0
:101F3000002383F31188DAE7C3689B695B68002B91
:101F4000D5D1C36F03B19847002384F87030CEE732
:101F5000024B0022C3E900339A607047A42C002092
:101F6000002382680374054B1B6899689142FBD279
:101F70005A6803604260106058607047A42C0020CB
:101F800008B5202383F31188037C032B05D0042B91
:101F90000DD02BB983F3118808BD436900221A6064
:101FA0004FF0FF334361FFF7DBFF0023F2E7D0E997
:101FB000003213605A60F3E7002382680374054B14
:101FC0001B6899689142FBD85A68036042601060B0
:101FD00058607047A42C0020054B196908741868D4
:101FE000026853601A60186101230374FEF7EEB9AA
:101FF000A42C00204B1C30B5044687B00A4D10D0ED
:102000002B6901A8094A00F025F92046FFF7E4FFF3
:10201000049B13B101A800F059F92B69586907B066
:1020200030BDFFF7D9FFF8E7A42C0020811F00087E
:1020300038B50C4D044641612B6981689A6891421C
:1020400003D8BDE83840FFF78BBF1846FFF7B4FF51
:1020500001232C61014623742046BDE83840FEF779
:10206000B5B900BFA42C0020044B1A681B69906806
:102070009B68984294BF002001207047A42C002048
:1020800010B5084C236820691A6854602260012248
:1020900023611A74FFF790FF01462069BDE81040E4
:1020A000FEF794B9A42C002008B5FFF7DDFF18B1A6
:1020B000BDE80840FFF7E4BF08BD0000FFF7E0BF40
:1020C000FEE7000010B50C4CFFF742FF00F0B4F83B
:1020D00080220A49204600F03BF8012344F8180CFE
:1020E000037400F09BFC002383F3118862B604485C
:1020F000BDE8104000F04CB8CC2C0020D8410008BE
:10210000E841000800F01CB9EFF3118020B9EFF3AB
:102110000583202282F311887047000010B530B982
:10212000EFF30584C4F3080414B180F3118810BDE3
:10213000FFF7BAFF84F31188F9E70000034A5168FA
:1021400053685B1A9842FBD8704700BF001000E04C
:1021500082600222028270478368A3F17C0243F806
:102160000C2C026943F83C2C426943F8382C074A8E
:1021700043F81C2CC268A3F1180043F8102C02226B
:1021800003F8082C002203F8072C7047E503000829
:1021900010B5202383F31188FFF7DEFF00210446EA
:1021A000FFF746FF002383F31188204610BD00008F
:1021B000024B1B6958610F20FFF70EBFA42C0020B3
:1021C000202383F31188FFF7F3BF000008B5014611
:1021D000202383F311880820FFF70CFF002383F3EB
:1021E000118808BD49B1064B42681B6918605A60E6
:1021F000136043600420FFF7FDBE4FF0FF307047CF
:10220000A42C00200368984206D01A68026050602F
:1022100018465961FFF7A4BE7047000038B5044660
:102220000D462068844200D138BD036823605C609D
:102230004561FFF795FEF4E7054B4FF0FF3103F1E1
:102240001402C3E905220022C3E90712704700BF48
:10225000A42C002070B51C4E05460C46C0E9032393
:1022600001F0B4FB334653F8142F9A420DD130627B
:102270000A2C2CBF00190A302A60C5E90124C6E9DE
:102280000555BDE8704001F08BBB316A431AE31875
:1022900038BF1C469368A34202D9081901F090FB8D
:1022A00073699A6894420CD85A68AC602B606A6073
:1022B00015609A685D60121B9A604FF0FF33F361FE
:1022C00070BDA41A1B68ECE7A42C002038B51B4C89
:1022D000636998420DD08168D0E9003213605A607A
:1022E0000022C2609A680A449A604FF0FF33E361AB
:1022F00038BD03682246002142F8143F93425A60D9
:10230000C16003D1BDE8384001F054BB9A688168D0
:10231000256A0A449A6001F059FB6369411B9A6877
:102320008A42E5D9AB181D1A206A092D98BF01F120
:102330000A02BDE83840104401F042BBA42C002042
:102340002DE9F041184C002704F11406656901F0ED
:102350003DFB236AAA68C11A8A4215D81344D5F8EE
:102360000C802362D5E9003213605A606369EF6024
:10237000B34201D101F01EFB87F311882869C047E1
:10238000202383F31188E1E76169B14209D0134446
:102390001B1ABDE8F0410A2B2CBFC0180A3001F00F
:1023A0000FBBBDE8F08100BFA42C002000207047C7
:1023B000FEE70000704700004FF0FF30704700005C
:1023C00002290CD0032904D00129074818BF002096
:1023D0007047032A05D8054800EBC200704704483F
:1023E00070470020704700BFCC4200083C2200200C
:1023F0008042000870B59AB005460846144601A907
:1024000000F0C2F801A8FEF74BFD431C0022C6B243
:102410005B001046C5E9003423700323023404F83E
:10242000013C01ABD1B202348E4201D81AB070BD6A
:1024300013F8011B013204F8010C04F8021CF1E747
:1024400008B5202383F311880348FFF767FA0023B8
:1024500083F3118808BD00BF602E002090F8803003
:1024600003F01F02012A07D190F881200B2A03D123
:102470000023C0E91D3315E003F06003202B08D1D1
:10248000B0F884302BB990F88120212A03D81F2A74
:1024900004D8FFF725BA222AEBD0FAE7034A4267AD
:1024A00007228267C3670120704700BF33220020E4
:1024B00007B5052917D8DFE801F019160319192007
:1024C000202383F31188104A01210190FFF7CEFAEF
:1024D000019802210D4AFFF7C9FA0D48FFF7EAF902
:1024E000002383F3118803B05DF804FB202383F3FA
:1024F00011880748FFF7B4F9F2E7202383F3118826
:102500000348FFF7CBF9EBE72042000844420008FC
:10251000602E002038B50C4D0C4C2A460C4904F1B5
:102520000800FFF767FF05F1CA0204F1100009492E
:10253000FFF760FF05F5CA7204F118000649BDE80F
:102540003840FFF757BF00BF384700203C2200202B
:10255000004200080A4200081542000870B504460F
:1025600008460D46FEF79CFCC6B2204601340378AF
:102570000BB9184670BD32462946FEF77DFC00288F
:10258000F3D10120F6E700002DE9F84F05460C468F
:10259000FEF786FC2C49C6B22846FFF7DFFF08B1DC
:1025A0000536F6B229492846FFF7D8FF08B110369C
:1025B000F6B2632E0DD8DFF89080DFF89090244FAC
:1025C000DFF894A0DFF894B02E7846B92670BDE805
:1025D000F88F29462046BDE8F84F01F0A9BD252E09
:1025E0002ED1072241462846FEF746FC70B9DBF89B
:1025F000003007350C3444F80C3CDBF8043044F868
:10260000083CDBF8083044F8043CDDE70822494682
:102610002846FEF731FC98B9A21C0E4B19780232FD
:102620000909C95D02F8041C13F8011B01F00F0130
:102630005345C95D02F8031CF0D118340835C3E7CF
:10264000013504F8016BBFE7EC42000815420008B1
:102650000143000800E8F11F0CE8F11FF4420008F4
:10266000BFF34F8F044B1A695107FCD1D3F81021E7
:102670005207F8D1704700BF0020005208B50D4B3B
:102680001B78ABB9FFF7ECFF0B4BDA68D10704D529
:102690000A4A5A6002F188325A60D3F80C21D207F4
:1026A00006D5064AC3F8042102F18832C3F8042192
:1026B00008BD00BF96490020002000522301674555
:1026C00008B5114B1B78F3B9104B1A69510703D5A4
:1026D000DA6842F04002DA60D3F81021520705D5DB
:1026E000D3F80C2142F04002C3F80C21FFF7B8FFE9
:1026F000064BDA6842F00102DA60D3F80C2142F0AE
:102700000102C3F80C2108BD9649002000200052A8
:102710000F289ABF00F58060400400207047000039
:102720004FF4003070470000102070470F2808B5A4
:102730000BD8FFF7EDFF00F500330268013204D13A
:1027400004308342F9D1012008BD0020FCE70000DD
:102750000F2870B5054645D8FFF7D6FC224CFFF789
:102760007FFF0646FFF78AFF4FF0FF33072D6361B7
:10277000C4F8143120D82361FFF772FF2B0243F015
:102780002403E360E36843F08003E36023695A07AE
:10279000FCD42846FFF764FF4FF40031FFF7B8FF81
:1027A00000F002F93046FFF78BFFFFF7B7FC284631
:1027B000BDE87040FFF7BABFC4F81031FFF750FF13
:1027C000A5F108031B0243F02403C4F80C31D4F82C
:1027D0000C3143F08003C4F80C31D4F810315B079E
:1027E000FBD4D6E7002070BD002000522DE9F84F41
:1027F00040EA020305460C461746D80602D00020E0
:10280000BDE8F88F27F01F07DFF8D4B0FFF736FFD9
:102810002744BC4203D10120FFF752FFF0E72022FA
:102820002946204601F074FC10B920352034F0E729
:102830002B4605F120021E68711CE0D104339A4238
:10284000F9D1FFF761FC05F17843234AB3F5801F06
:10285000224B28BF9A4603F1040338BF9046A2F1E9
:10286000080228BF9846A3F108033ABF9146DA460A
:102870009946FFF7F5FEC8F80060A5EB040CD9F8FF
:10288000002004F11C0142F00202C9F80020221FBE
:10289000DAF8006016F00506FAD152F8043F8A42D1
:1028A0004CF80230F4D1BFF34F8FFFF7D9FE4FF051
:1028B000FF32C8F80020D9F8002022F00202C9F83F
:1028C0000020FFF72BFC20222146284601F020FCA7
:1028D0000028AAD030469FE7142000521021005251
:1028E0001020005210B5084C237828B11BB9FFF70F
:1028F000C5FE0123237010BD002BFCD02070BDE865
:102900001040FFF7DDBE00BF964900200244074B90
:10291000D2B210B5904200D110BD441C00B253F8A1
:10292000200041F8040BE0B2F4E700BF504000582B
:102930000E4B30B51C6F240405D41C6F1C671C6F34
:1029400044F400441C670A4C02442368D2B243F4A6
:1029500080732360074B904200D130BD441C51F876
:10296000045B00B243F82050E0B2F4E700440258A0
:10297000004802585040005807B5012201A9002024
:10298000FFF7C4FF019803B05DF804FB13B50446DC
:10299000FFF7F2FFA04205D0012201A90020019417
:1029A000FFF7C6FF02B010BD0144BFF34F8F064BC7
:1029B000884204D3BFF34F8FBFF36F8F7047C3F8C4
:1029C0005C022030F4E700BF00ED00E0002070471B
:1029D000034B1A681AB9034AD2F8D0241A60704718
:1029E000984900200040025808B5FFF7F1FF024B5C
:1029F0001868C0F3806008BD98490020EFF3098390
:102A0000054968334A6B22F001024A6383F309885F
:102A1000002383F31188704700EF00E0202080F34B
:102A2000118862B60D4B0E4AD96821F4E0610904A1
:102A3000090C0A430B49DA60D3F8FC2042F080729B
:102A4000C3F8FC20084AC2F8B01F116841F0010128
:102A500011601022DA7783F82200704700ED00E061
:102A60000003FA0555CEACC5001000E0202310B5D8
:102A700083F311880E4B5B6813F4006314D0F1EEFE
:102A8000103AEFF309844FF08073683CE361094B1F
:102A9000DB6B236684F30988FFF7E6FA10B1064B77
:102AA000A36110BD054BFBE783F31188F9E700BF75
:102AB00000ED00E000EF00E0F7030008FA03000873
:102AC00070B5BFF34F8FBFF36F8F1A4A0021C2F862
:102AD0005012BFF34F8FBFF36F8F536943F400332E
:102AE0005361BFF34F8FBFF36F8FC2F88410BFF3F2
:102AF0004F8FD2F8803043F6E074C3F3C900C3F3BC
:102B00004E335B0103EA0406014646EA817501394A
:102B1000C2F86052F9D2203B13F1200FF2D1BFF37B
:102B20004F8F536943F480335361BFF34F8FBFF32B
:102B30006F8F70BD00ED00E0FEE700000A4B0B4810
:102B40000B4A90420BD30B4BC11EDA1C121A22F017
:102B500003028B4238BF00220021FEF7A9B953F8C7
:102B6000041B40F8041BECE7E44400086C4B002015
:102B70006C4B00206C4B00207047000070B5D0E912
:102B8000244300224FF0FF359E6804EB42135101AD
:102B9000D3F80009002805DAD3F8000940F0804096
:102BA000C3F80009D3F8000B002805DAD3F8000BAE
:102BB00040F08040C3F8000B013263189642C3F81E
:102BC0000859C3F8085BE0D24FF00113C4F81C3871
:102BD00070BD000000EB8103D3F80CC02DE9F04379
:102BE000DCF814204E1CD0F89050D2F800E005EB31
:102BF000063605EB4118506870450AD30122D5F816
:102C0000343802FA01F123EA0101C5F83418BDE8AD
:102C1000F083AEEB0003BCF81040A34228BF23466C
:102C2000D8F81849A4B2B3EB840FF0D89468A4F193
:102C3000040959F8047F3760A4EB09071F44042FE7
:102C4000F7D81C44034494605360D4E7890141F0F1
:102C50002001016103699B06FCD41220FFF76EBAC4
:102C600010B50A4C2046FEF7DFFE094BC4F8903041
:102C7000084BC4F89430084C2046FEF7D5FE074BAD
:102C8000C4F89030064BC4F8943010BD9C49002025
:102C90000000084038430008384A00200000044083
:102CA0004443000870B503780546012B5DD1494BBC
:102CB000D0F89040984259D1474B0E216520D3F867
:102CC000D82042F00062C3F8D820D3F8002142F0A7
:102CD0000062C3F80021D3F80021D3F8802042F02D
:102CE0000062C3F88020D3F8802022F00062C3F88D
:102CF0008020D3F8803000F071FC384BE360384B13
:102D0000C4F800380023D5F89060C4F8003EC02312
:102D100023604FF40413A3633369002BFCDA01230F
:102D20000C203361FFF70AFA3369DB07FCD4122069
:102D3000FFF704FA3369002BFCDA00262846A66068
:102D4000FFF71CFF6B68C4F81068DB68C4F81468F0
:102D5000C4F81C68002B3AD1224BA3614FF0FF331B
:102D60006361A36843F00103A36070BD1E4B9842EA
:102D7000C8D1194B0E214D20D3F8D82042F0007253
:102D8000C3F8D820D3F8002142F00072C3F8002124
:102D9000D3F80021D3F8802042F00072C3F88020DD
:102DA000D3F8802022F00072C3F88020D3F880206E
:102DB000D3F8D82022F08062C3F8D820D3F80021BD
:102DC00022F08062C3F80021D3F8003193E7074B6B
:102DD000C3E700BF9C490020004402584014004053
:102DE00003002002003C30C0384A0020083C30C0BC
:102DF000F8B5D0F89040054600214FF00066204617
:102E0000FFF724FFD5F8941000234FF001128F68CC
:102E10004FF0FF30C4F83438C4F81C2804EB4312D8
:102E200001339F42C2F80069C2F8006BC2F808097A
:102E3000C2F8080BF2D20B68D5F89020C5F898308C
:102E4000636210231361166916F01006FBD112207D
:102E5000FFF774F9D4F8003823F4FE63C4F800389F
:102E6000A36943F4402343F01003A3610923C4F88A
:102E70001038C4F814380B4BEB604FF0C043C4F863
:102E8000103B094BC4F8003BC4F81069C4F8003982
:102E9000D5F8983003F1100243F48013C5F8982058
:102EA000A362F8BD1443000840800010D0F89020C1
:102EB00090F88A10D2F8003823F4FE6343EA011335
:102EC000C2F80038704700002DE9F84300EB810399
:102ED000D0F890500C468046DA680FFA81F9480124
:102EE000166806F00306731E022B05EB41134FF024
:102EF000000194BFB604384EC3F8101B4FF0010117
:102F000004F1100398BF06F1805601FA03F39169AA
:102F100098BF06F5004600293AD0578A04F15801B7
:102F2000374349016F50D5F81C180B430021C5F8F1
:102F30001C382B180127C3F81019A7405369611ECC
:102F40009BB3138A928B9B08012A88BF5343D8F8FE
:102F50009820981842EA034301F140022146C8F83C
:102F60009800284605EB82025360FFF76FFE08EBDE
:102F70008900C3681B8A43EA845348341E436401B2
:102F80002E51D5F81C381F43C5F81C78BDE8F883CE
:102F900005EB4917D7F8001B21F40041C7F8001BC7
:102FA000D5F81C1821EA0303C0E704F13F030B4ADC
:102FB0002846214605EB83035A60FFF747FE05EBE1
:102FC0004910D0F8003923F40043C0F80039D5F88F
:102FD0001C3823EA0707D7E700800010000400022E
:102FE000D0F894201268C0F89820FFF7C7BD000001
:102FF0005831D0F8903049015B5813F4004004D0A8
:1030000013F4001F0CBF0220012070474831D0F894
:10301000903049015B5813F4004004D013F4001FB2
:103020000CBF02200120704700EB8101CB68196AB8
:103030000B6813604B6853607047000000EB81031E
:1030400030B5DD68AA691368D36019B9402B84BF15
:10305000402313606B8A1468D0F890201C4402EB64
:103060004110013C09B2B4FBF3F46343033323F092
:10307000030343EAC44343F0C043C0F8103B2B684A
:1030800003F00303012B0ED1D2F8083802EB4110F4
:1030900013F4807FD0F8003B14BF43F0805343F01B
:1030A0000053C0F8003B02EB4112D2F8003B43F062
:1030B0000443C2F8003B30BD2DE9F041D0F89060E8
:1030C00005460C4606EB4113D3F8087B3A07C3F8D4
:1030D000087B08D5D6F814381B0704D500EB81030C
:1030E000DB685B689847FA071FD5D6F81438DB070A
:1030F0001BD505EB8403D968CCB98B69488A5A681B
:10310000B2FBF0F600FB16228AB91868DA68904222
:103110000DD2121AC3E90024202383F3118821461B
:103120002846FFF78BFF84F31188BDE8F081012367
:1031300003FA04F26B8923EA02036B81CB68002B4C
:10314000F3D021462846BDE8F041184700EB810343
:103150004A0170B5DD68D0F890306C692668E66089
:1031600056BB1A444FF40020C2F810092A6802F036
:103170000302012A0AB20ED1D3F8080803EB421465
:1031800010F4807FD4F8000914BF40F0805040F064
:103190000050C4F8000903EB4212D2F8000940F0D5
:1031A0000440C2F800090122D3F8340802FA01F100
:1031B0000143C3F8341870BD19B9402E84BF4020B4
:1031C000206020681A442E8A8419013CB4FBF6F46E
:1031D00040EAC44040F00050C6E700002DE9F0414D
:1031E000D0F8906004460D4606EB4113D3F80879F9
:1031F000C3F80879FB071CD5D6F81038DA0718D5BC
:1032000000EB8103D3F80CC0DCF81430D3F800E0F5
:10321000DA6896451BD2A2EB0E024FF000081A6046
:10322000C3F80480202383F31188FFF78FFF88F30E
:1032300011883B0618D50123D6F83428AB40134239
:1032400012D029462046BDE8F041FFF7C3BC012358
:1032500003FA01F2038923EA02030381DCF8083050
:10326000002BE6D09847E4E7BDE8F0812DE9F84F60
:10327000D0F8905004466E69AB691E4016F4805831
:103280006E6103D0BDE8F84FFEF73EBC002E12DAA7
:10329000D5F8003E9F0705D0D5F8003E23F0030384
:1032A000C5F8003ED5F80438204623F00103C5F8E0
:1032B0000438FEF755FC300505D52046FFF75EFCC7
:1032C0002046FEF73DFCB1040CD5D5F8083813F0C4
:1032D000060FEB6823F470530CBF43F4105343F410
:1032E000A053EB60320704D56368DB680BB120465E
:1032F0009847F30200F1BA80B70226D5D4F890902F
:1033000000274FF0010A09EB4712D2F8003B03F403
:103310004023B3F5802F11D1D2F8003B002B0DDAFA
:1033200062890AFA07F322EA0303638104EB870345
:10333000DB68DB6813B13946204698470137D4F87B
:103340009430FFB29B689F42DDD9F00619D5D4F8BE
:103350009000026AC2F30A1702F00F0302F4F0129F
:10336000B2F5802F00F0CC80B2F5402F09D104EBEC
:103370008303002200F58050DB681B6A974240F00F
:10338000B2803003D5F8185835D5E90303D50021AC
:103390002046FFF791FEAA0303D501212046FFF73F
:1033A0008BFE6B0303D502212046FFF785FE2F031A
:1033B00003D503212046FFF77FFEE80203D5042151
:1033C0002046FFF779FEA90203D505212046FFF725
:1033D00073FE6A0203D506212046FFF76DFE2B021D
:1033E00003D507212046FFF767FEEF0103D508212B
:1033F0002046FFF761FE700340F1A980E90703D57D
:1034000000212046FFF7EAFEAA0703D50121204646
:10341000FFF7E4FE6B0703D502212046FFF7DEFE2F
:103420002F0703D503212046FFF7D8FEEE0603D56C
:1034300004212046FFF7D2FEA80603D50521204629
:10344000FFF7CCFE690603D506212046FFF7C6FE2E
:103450002A0603D507212046FFF7C0FEEB0576D5E7
:1034600020460821BDE8F84FFFF7B8BED4F8909089
:1034700000274FF0010AD4F894305FFA87FB9B686D
:103480009B453FF639AF09EB4B13D3F8002902F403
:103490004022B2F5802F24D1D3F80029002A20DA67
:1034A000D3F8002942F09042C3F80029D3F800294C
:1034B000002AFBDB5946D4F89000FFF7C7FB2289AE
:1034C0000AFA0BF322EA0303238104EB8B03DB6884
:1034D0009B6813B159462046984759462046FFF746
:1034E00079FB0137C7E7910701D1D0F80080072A9F
:1034F00002F101029CBF03F8018B4FEA18283DE757
:1035000004EB830300F58050DA68D2F818C0DCF8C9
:103510000820DCE9001CA1EB0C0C00218F4208D133
:10352000DB689B699A683A449A605A683A445A60E0
:1035300027E711F0030F01D1D0F800808C4501F18D
:10354000010184BF02F8018B4FEA1828E6E7BDE8C5
:10355000F88F000008B50348FFF788FEBDE8084073
:10356000FFF784BA9C49002008B50348FFF77EFEA8
:10357000BDE80840FFF77ABA384A0020D0F890300A
:1035800003EB4111D1F8003B43F40013C1F8003BB9
:1035900070470000D0F8903003EB4111D1F80039AA
:1035A00043F40013C1F8003970470000D0F89030A0
:1035B00003EB4111D1F8003B23F40013C1F8003BA9
:1035C00070470000D0F8903003EB4111D1F800397A
:1035D00023F40013C1F8003970470000090100F11D
:1035E0006043012203F56143C9B283F8001300F080
:1035F0001F039A4043099B0003F1604303F56143B5
:10360000C3F880211A60704730B50433039C0172FF
:10361000002104FB0325C160C0E90653049B03633A
:10362000059BC0E90000C0E90422C0E90842C0E9E6
:103630000A11436330BD00000022416AC260C0E944
:103640000411C0E90A226FF00101FEF7E7BD000096
:10365000D0E90432934201D1C2680AB9181D7047FB
:1036600000207047036919600021C2680132C260FE
:10367000C269134482699342036124BF436A0361B0
:10368000FEF7C0BD38B504460D46E3683BB162693C
:103690000020131D1268A3621344E36207E0237A3B
:1036A00033B929462046FEF79DFD0028EDDA38BDE6
:1036B0006FF00100FBE70000C368C269013BC36013
:1036C0004369134482699342436124BF436A43615F
:1036D00000238362036B03B11847704770B5202342
:1036E000044683F31188866A3EB9FFF7CBFF05468F
:1036F00018B186F31188284670BDA36AE26A13F8F0
:10370000015B9342A36202D32046FFF7D5FF00235B
:1037100083F31188EFE700002DE9F84F04460E46C9
:10372000174698464FF0200989F311880025AA46CC
:10373000D4F828B0BBF1000F09D141462046FFF76D
:10374000A1FF20B18BF311882846BDE8F88FD4E99A
:103750000A12A7EB050B521A934528BF9346BBF1FB
:10376000400F1BD9334601F1400251F8040B91423E
:1037700043F8040BF9D1A36A403640354033A362C5
:10378000D4E90A239A4202D32046FFF795FF8AF331
:103790001188BD42D8D289F31188C9E730465A460C
:1037A000FDF760FBA36A5E445D445B44A362E7E708
:1037B00010B5029C0433017204FB0321C460C0E90C
:1037C00006130023C0E90A33039B0363049BC0E98B
:1037D0000000C0E90422C0E90842436310BD0000B4
:1037E000026A6FF00101C260426AC0E9042200224D
:1037F000C0E90A22FEF712BDD0E904239A4201D1A2
:10380000C26822B9184650F8043B0B60704700208C
:1038100070470000C3680021C2690133C360436977
:10382000134482699342436124BF436A4361FEF7B4
:10383000E9BC000038B504460D46E3683BB1236996
:1038400000201A1DA262E2691344E36207E0237AB2
:1038500033B929462046FEF7C5FC0028EDDA38BD0D
:103860006FF00100FBE7000003691960C268013ACC
:10387000C260C269134482699342036124BF436AF0
:10388000036100238362036B03B118477047000094
:1038900070B520230D460446114683F31188866ACD
:1038A0002EB9FFF7C7FF10B186F3118870BDA36A68
:1038B0001D70A36AE26A01339342A36204D3E169F3
:1038C00020460439FFF7D0FF002080F31188EDE790
:1038D0002DE9F84F04460D46904699464FF0200AD0
:1038E0008AF311880026B346A76A4FB94946204695
:1038F000FFF7A0FF20B187F311883046BDE8F88FAD
:10390000D4E90A073A1AA8EB0607974228BF1746D8
:10391000402F1BD905F1400355F8042B9D4240F878
:10392000042BF9D1A36A40364033A362D4E90A23B9
:103930009A4204D3E16920460439FFF795FF8BF3DF
:1039400011884645D9D28AF31188CDE729463A46EF
:10395000FDF788FAA36A3D443E443B44A362E5E791
:10396000D0E904239A4217D1C3689BB1836A8BB113
:10397000043B9B1A0ED01360C368013BC360C3694C
:103980001A4483699A42026124BF436A0361002397
:1039900083620123184670470023FBE700F0DAB882
:1039A000034B002258631A610222DA60704700BF9D
:1039B000000C0040014B0022DA607047000C004010
:1039C000014B5863704700BF000C0040014B586A20
:1039D000704700BF000C00404B6843608B688360F9
:1039E000CB68C3600B6943614B6903628B694362B7
:1039F0000B6803607047000008B53C4B40F2FF7154
:103A00003B48D3F888200A43C3F88820D3F888209D
:103A100022F4FF6222F00702C3F88820D3F888203E
:103A2000D3F8E0200A43C3F8E020D3F808210A4382
:103A3000C3F808212F4AD3F808311146FFF7CCFF0D
:103A400000F5806002F11C01FFF7C6FF00F5806001
:103A500002F13801FFF7C0FF00F5806002F1540168
:103A6000FFF7BAFF00F5806002F17001FFF7B4FFC5
:103A700000F5806002F18C01FFF7AEFF00F5806079
:103A800002F1A801FFF7A8FF00F5806002F1C40170
:103A9000FFF7A2FF00F5806002F1E001FFF79CFF55
:103AA00000F5806002F1FC01FFF796FF02F58C71D2
:103AB00000F58060FFF790FF00F000F90E4BD3F89F
:103AC000902242F00102C3F89022D3F8942242F0EF
:103AD0000102C3F894220522C3F898204FF06052E7
:103AE000C3F89C20054AC3F8A02008BD0044025832
:103AF000000002585043000800ED00E01F000803DA
:103B000008B500F0E5FAFEF7DDFA0F4BD3F8DC203C
:103B100042F04002C3F8DC20D3F8042122F0400236
:103B2000C3F80421D3F80431084B1A6842F00802A4
:103B30001A601A6842F004021A60FEF749FFBDE8F5
:103B40000840FEF7E7BC00BF0044025800180248D6
:103B500070470000114BD3F8E82042F00802C3F888
:103B6000E820D3F8102142F00802C3F810210C4AD3
:103B7000D3F81031D36B43F00803D363C722094B4A
:103B80009A624FF0FF32DA6200229A615A63DA6079
:103B90005A6001225A611A60704700BF00440258FF
:103BA0000010005C000C0040094A08B51169D36898
:103BB0000B40D9B29B076FEA0101116107D52023A1
:103BC00083F31188FEF79EFA002383F3118808BD62
:103BD000000C0040384B4FF0FF31D3F88020C3F881
:103BE0008010D3F880200022C3F88020D3F8800012
:103BF000D3F88400C3F88410D3F88400C3F8842079
:103C0000D3F88400D86F40F0FF4040F4FF0040F448
:103C10003F5040F03F00D867D86F20F0FF4020F4BD
:103C2000FF0020F43F5020F03F00D867D86FD3F852
:103C300088006FEA40506FEA5050C3F88800D3F80C
:103C40008800C0F30A00C3F88800D3F88800D3F8CE
:103C50009000C3F89010D3F89000C3F89020D3F8E8
:103C60009000D3F89400C3F89410D3F89400C3F8EC
:103C70009420D3F89400D3F89800C3F89810D3F8A0
:103C80009800C3F89820D3F89800D3F88C00C3F8B4
:103C90008C10D3F88C00C3F88C20D3F88C00D3F8A8
:103CA0009C00C3F89C10D3F89C10C3F89C20D3F858
:103CB0009C3000F0DDB900BF00440258614B012286
:103CC000C3F80821604BD3F8F42042F00202C3F895
:103CD000F420D3F81C2142F00202C3F81C21022276
:103CE000D3F81C31594BDA605A689104FCD5584A14
:103CF0001A6001229A60574ADA6000221A614FF472
:103D000040429A61514B9A699204FCD51A6842F478
:103D100080721A604C4B1A6F12F4407F04D04FF43B
:103D200080321A6700221A671A6842F001021A608C
:103D3000454B1A685007FCD500221A611A6912F027
:103D40003802FBD1012119604FF0804159605A6758
:103D5000414ADA62414A1A611A6842F480321A60B2
:103D6000394B1A689103FCD51A6842F480521A60E4
:103D70001A689204FCD53A4A3A499A6200225A6378
:103D800019633949DA6399635A64384A1A64384ABC
:103D9000DA621A6842F0A8521A602B4B1A6802F0D5
:103DA0002852B2F1285FF9D148229A614FF4886213
:103DB000DA6140221A622F4ADA644FF080521A65A3
:103DC0002D4A5A652D4A9A6532232D4A136013688D
:103DD00003F00F03022BFAD11B4B1A6942F00302C6
:103DE0001A611A6902F03802182AFAD1D3F8DC20D5
:103DF00042F00052C3F8DC20D3F8042142F0005214
:103E0000C3F80421D3F80421D3F8DC2042F0804227
:103E1000C3F8DC20D3F8042142F08042C3F8042127
:103E2000D3F80421D3F8DC2042F00042C3F8DC20B0
:103E3000D3F8042142F00042C3F80421D3F804313E
:103E4000704700BF008000510044025800480258EB
:103E500000C000F0020000010000FF01008890088F
:103E600032206000630209011D02040047040508B6
:103E7000FD0BFF01200000200010E0000001010008
:103E8000002000524FF0B04208B5D2F8883003F05D
:103E90000103C2F8883023B1044A13680BB150689B
:103EA0009847BDE80840FEF7E1BD00BFEC4A00209E
:103EB0004FF0B04208B5D2F8883003F00203C2F8E0
:103EC000883023B1044A93680BB1D0689847BDE8A5
:103ED0000840FEF7CBBD00BFEC4A00204FF0B042D7
:103EE00008B5D2F8883003F00403C2F8883023B153
:103EF000044A13690BB150699847BDE80840FEF7C2
:103F0000B5BD00BFEC4A00204FF0B04208B5D2F872
:103F1000883003F00803C2F8883023B1044A93695B
:103F20000BB1D0699847BDE80840FEF79FBD00BFC0
:103F3000EC4A00204FF0B04208B5D2F8883003F0C8
:103F40001003C2F8883023B1044A136A0BB1506AD7
:103F50009847BDE80840FEF789BD00BFEC4A002045
:103F60004FF0B04310B5D3F8884004F47872C3F82A
:103F70008820A30604D5124A936A0BB1D06A9847E9
:103F8000600604D50E4A136B0BB1506B984721069F
:103F900004D50B4A936B0BB1D06B9847E20504D55F
:103FA000074A136C0BB1506C9847A30504D5044A1B
:103FB000936C0BB1D06C9847BDE81040FEF756BD2E
:103FC000EC4A00204FF0B04310B5D3F8884004F419
:103FD0007C42C3F88820620504D5164A136D0BB1E4
:103FE000506D9847230504D5124A936D0BB1D06DDF
:103FF0009847E00404D50F4A136E0BB1506E9847F2
:10400000A10404D50B4A936E0BB1D06E984762049D
:1040100004D5084A136F0BB1506F9847230404D599
:10402000044A936F0BB1D06F9847BDE81040FEF77C
:104030001DBD00BFEC4A002008B50348FDF706F996
:10404000BDE80840FEF712BDCC23002008B50348A8
:10405000FDF7FCF8BDE80840FEF708BD3824002055
:1040600008B5FFF7A1FDBDE80840FEF7FFBC000062
:10407000062108B50846FFF7B1FA06210720FFF729
:10408000ADFA06210820FFF7A9FA06210920FFF75B
:10409000A5FA06210A20FFF7A1FA06211720FFF74B
:1040A0009DFA06212820FFF799FA09217A20FFF7C7
:1040B00095FA07213220FFF791FA0C212620FFF70D
:1040C0008DFA0C215220BDE80840FFF787BA0000A6
:1040D00008B5FFF77FFD00F00DF8FDF7C9FAFDF711
:1040E000A1FCFDF773FBFFF733FDBDE80840FFF7C8
:1040F00055BC00000023054A19460133102BC2E9C4
:10410000001102F10802F8D1704700BFEC4A00200C
:1041100010B501390244904201D1002005E0037836
:1041200011F8014FA34201D0181B10BD0130F2E776
:10413000034611F8012B03F8012B002AF9D170472F
:1041400053544D333248373F3F3F0053544D333281
:10415000483734332F37353300000000CC2300209C
:10416000602E00200096000000000000000000000B
:10417000000000000000000000000000000000003F
:104180003916000825160008611600084D160008AB
:104190005916000845160008311600081D160008BB
:1041A0006D160008000000004917000835170008C8
:1041B000711700085D1700086917000855170008F7
:1041C000411700082D1700087D17000800000000A7
:1041D00001000000000000006D61696E0000000039
:1041E00069646C6500000000E0410008E82C0020D4
:1041F000602E002001000000C12000080000000027
:104200004172647550696C6F740025424F4152448D
:10421000252D424C002553455249414C25000000B4
:10422000020000000000000069190008D919000808
:10423000400040000847002018470020020000000E
:10424000000000000300000000000000211A000828
:1042500000000000100000002847002000000000BF
:1042600001000000000000009C4900200101020044
:10427000B1240008C12300085D240008412400087F
:10428000430000008842000809024300020100C008
:10429000320904000001020201000524001001059A
:1042A00024010001042402020524060001070582FE
:1042B000030800FF09040100020A000000070501CD
:1042C00002400000070581024000000012000000CB
:1042D000D4420008120110010200004009124157A7
:1042E00000020102030100000403090425424F41BA
:1042F000524425006C756D696E6F75736265653526
:104300000030313233343536373839414243444551
:104310004600000000000000751B00082D1E00086C
:10432000D91E000840004000D44A0020D44A002092
:1043300001000000E44A002080000000400100006D
:104340000800000000010000000400000800000058
:104350000000802A00000000AAAAAAAA00000024E7
:10436000FFFF00000000000000A00A000001400064
:1043700000000000AAAAAAAA00010000FFFF000096
:1043800000000000000000001000004000000000DD
:10439000AAAAAAAA10000040FFFF00000000000027
:1043A000000000000068000000000000AAAAAAAAFD
:1043B00000540000FFFF0000000070070000000034
:1043C0000080024000000000AAAAAAAA0040014002
:1043D000FFFF000000000070070000000000000068
:1043E00000000000AAAAAAAA00000000FFFF000027
:1043F00000000000000000000000000000000000BD
:10440000AAAAAAAA00000000FFFF00000000000006
:10441000000000000000000000000000AAAAAAAAF4
:1044200000000000FFFF000000000000000000008E
:104430000000000000000000AAAAAAAA00000000D4
:10444000FFFF00000000000000000000000000006E
:1044500000000000AAAAAAAA00000000FFFF0000B6
:10446000000000000000000000000000000000004C
:10447000AAAAAAAA00000000FFFF00000000000096
:104480000000000000000000050400000000000023
:1044900000001E0000000000FF00000000000000FF
:1044A000404100083F000000500400004B4100085C
:1044B0003F00000000960000000008009600000089
:1044C0000008000004000000E842000800000000AE
:1044D00000000000000000000000000000000000DC
:0444E00000000000D8
:00000001FF
